:03000000021B5C84
:0C1B5C0078FFE4F6D8FD7581D102003658
:0100190022C4
:061863008B318A3289334B
:10186900756F027F481219CC121BA8EF20E0F9AB63
:1018790031AA32A93312074F7877E6FE08E6FDED63
:01188900FF5F
:01188A00223B
:100F5F0043525354005341564500434647002D3EDC
:100F6F0053320052415445434C5220554E4954423E
:100F7F004C4E4B5452494754524556535452545366
:100F8F00544F505A45524F44464C54534156455274
:100F9F00535420535720202E3235203173202032C6
:100FAF00732020357320203130732033307320317C
:100FBF006D2020326D2020356D202031306D203393
:100FCF00306D2031682020326820203468202000C6
:100FDF000000010004000800140028007800F00150
:100FEF00E004B009601C2038407080E10046656560
:100FFF0074596172644D6574724F6666204F6E202E
:10100F00204E6F2020596573204F66662054696DFE
:10101F0065416C7420547269674F66662054696D20
:10102F0065416C74204F6666205472696750777201
:05103F00205265632052
:10188B0025E024DEF582E4340FF583220533E533BE
:10189B00C394022208F608F608F62275F004A42475
:0518AB0008F974102291
:10145D00789776AB0876CD087600087604E408F622
:10146D0008760108F60876FA08764012189F08F6F5
:10147D0078A5760A08763C08F608761408F60876FC
:10148D000F12189F7BFF7A0F795F1217AA7F051233
:05149D0016D702180D36
:1019E70075731D7574C012170D7898E664CD700471
:0919F70018E664AB600312145DF4
:011A000022C3
:0D1B2400C2AF7DC07C1DE4FF121AA1D2AF3C
:011B31002291
:10170D007540FF85734185744275430075440075BE
:10171D004597E4FFAB40AA41A9428F827583001221
:10172D000722AB43AA44A9458F8275830012076136
:04173D000FBF18E0E2
:011741002285
:10180D007D01E4FF1219567BFF7A0F79641217AA36
:10181D00121B24C2AF7F977B187DC07C1D121AABA3
:0D182D00D2AF7F021216D7E4FDFF0219565C
:10095F00E4F5317BFF7A0F79691217AA7F0512161A
:10096F00D7A297829650FAA2969217A2979218E55D
:10097F003175F004A42472F9740F35F0FA7BFF126D
:10098F0017AA7F051216D7853132E4F5337BFF7A2C
:10099F000F796D1217AAE531B4090050779009B39A
:1009AF00F82828730209CE020A230209EF0209F779
:1009BF000209FB020A03020A0B020A13020A1B7F37
:1009CF0001EF12188B7899E6FC08E6FD7401936D20
:1009DF007003E4936C70028F330FBF0FE4020AA60B
:1009EF00789BE6F533020ACC789C800278A4E6F572
:1009FF0033020AE678A3E6F533020B0D78ABE6F582
:100A0F0033020B2A78ACE6F533020B4778ADE6F5E7
:100A1F0033020B64E5316532600302097EA21730A1
:100A2F009601B35013A296921730960C0531E5310B
:100A3F00C3940C4003E4F531A218309701B350D49E
:100A4F00A29792183097CDE531B40C0050C6900A9A
:100A5F0064F8282873020A88020AB4020ABA020A42
:100A6F00D8020AEC020AFF020B18020B35020B52D6
:100A7F00020B78020B7E020B840533E533C3940F10
:100A8F004003753301E53312188BE493FF74019320
:100A9F007899CFF608EFF6E53375F004A424A2F9A0
:100AAF00740F020B6D121318020A230533E533C3BB
:100ABF0094034003E4F533789BA633E53375F004D4
:100ACF00A424FCF9740F020B6D1218974003E4F580
:100ADF0033789CA633E5331218A6020B6D121897C4
:100AEF004003E4F53378A4A633E5331218A6806EDD
:100AFF001218974003E4F53378A3A633E53375F066
:100B0F0004A42410F9741080550533E533C39404FD
:100B1F004003E4F53378ABA633E53375F004A42432
:100B2F0018F9741080380533E533C394034003E498
:100B3F00F53378ACA633E53375F004A42428F974A3
:100B4F0010801B0533E533C394044003E4F5337879
:100B5F00ADA633E53375F004A42434F9741035F0E1
:100B6F00FA7BFF1217AA020A2312145D020A23123C
:0B0B7F00180D020A2343A208020A23FB
:0A1B74004552415300444F4E450016
:10199200E4D3FCFD7B80FAF9F80208C07899E6F5F9
:0D19A2005708E6F55822E568AE6778062282
:1011F900C215C216E4F532F533AE32AF3312199285
:10120900401CE53164816016AF33AE321217DC122F
:101219001A8D8F310533E53370DF053280DBE53117
:10122900B48108E533153370021532AE32AF33E4B9
:10123900C3121994700CD215121B40E4F567F568B6
:101249008007853267853368E4F569F56A755680E4
:0312590012199EC9
:01125C00226F
:0417DC008F828E83E7
:1017E0001219924027E582AE837806C333CE33CEFA
:1017F000D8F9FD756F02EE7877F6CFEDCFEF08F6EA
:0C1800007F50121A34121BA8EF20E0F9F0
:01180C0022B9
:031A0100CDEFCD59
:101A0400756F02EE7877F6ED08F67F50121A3412ED
:061A14001BA8EF20E0F921
:011A1A0022A9
:101A8D00756F017F501219CC121BA8EF20E0F97869
:031A9D0077E6FFEA
:011AA0002223
:101A7800121A01E4FFFE0FBF00010EBE0FF8BFA04F
:041A8800F5121A8DAC
:011A8C002237
:06174200CBEFCBCAEECA9A
:10174800301503301627756F03EA7877F6EB08F63D
:1017580008EDF67F50121A34121BA8EF20E0F9E4C6
:0D176800FFFE0FBF00010EBE0FF8BFA0F581
:011775002251
:10156F00753400753500753656E4F5331219A8C376
:10157F0033CE33CED8F97C002533FFEC3EFEAB34AF
:10158F00AA35A936853382758300120722FD1217FB
:10159F00420533E533C3940640D2756900756A0678
:0115AF002219
:10110A008E318F321219A8C333CE33CED8F9256A5D
:10111A00FFE5693EFEEEC0E0EFC0E0E531FDD0E05C
:10112A00FFD0E0FE121742056AE56A7002056912ED
:10113A0019A8C333CE33CED8F9256AFFE5693EFE36
:10114A00AD32121742056AE56A70020569055AE569
:10115A005A70020559C3E56A9440E569940040173C
:10116A00E4F569F56A0568E56870020567AE67FF28
:08117A001219925002D2152255
:10131800E4F569F56A7BFF7A1B79741217AAD2166D
:10132800E4F540F541AE40AF411219924021E54144
:10133800AE407806C333CE33CED8F9F56A8E697DD0
:1013480081FF1217420541E54170DA054080D6C297
:10135800167BFF7A1B79791217AAE4F567F568F509
:0513680069F56AC215E1
:01136D00225D
:1012C100E4F540F541F542F543AE42AF43121992C0
:1012D1004044E5416481603EAF43AE421217DC12E7
:1012E1001A8D8F41E54164807022AF400540FCFDBD
:1012F100FEFBFAF9120D367F2C120016AE42AF43F7
:10130100E4FCFDFBFAF9120D36121B910543E5438E
:0613110070B7054280B335
:0113170022B3
:0214A2008F4079
:1014A400E4F541F542F543F544AE43AF44121992D5
:1014B4004030E5426481602AAF44AE431217DC1227
:1014C4001A8D8F42E542B4800FE54165407007AF45
:1014D40044AE430217DC05410544E54470CB0543A3
:0214E40080C7BF
:0114E60022E3
:1016670012199E78A4E6F55BE4F559F55A12156F41
:1016770085676B85686C7F0112125D30021178A651
:10168700E6FF7E007C007D641207838E638F6430E3
:081697000505C205121A6222CA
:10169F00856731856832E56A456960080532E5324C
:1016AF0070020531856B67856C6812156F85316720
:1016BF00853268AE31AF321219925007E4F567F5F3
:0816CF0068D2157F0202125DD2
:101AA100740478FF769612FF0322740078FF76960D
:041AB10012FF0322FB
:0300330002104474
:0D104400C0E0C0F0C083C082C0D075D008ED
:10105100E5D954F8FF120939107E08107E10108D61
:101061001810A820108F2810A83010AA3810B040EE
:1010710010A84810C95010E658000010F48572DA23
:10108100C2DDC2DC7570007571008070800EE56F85
:10109100700280560571E571700205701200268F8D
:1010A100DAC2DDC2DC80558016D2DDC2DC804DC2E1
:1010B100DDC2DCE56F7004C2DA8041D2DA803DC264
:1010C100DDD2DC756D048034AFDA121B680571E581
:1010D1007170020570C2DDC2DCE56F7004C2DA8096
:1010E1001BD2DA8017AFDA121B68C2DDD2DC756D54
:0E10F100028009756D04C2DDC2DCD2DAC2DBFA
:0B10FF00D0D0D082D083D0F0D0E032FF
:10183A0043910C43920CE4F5DBEF25E0F5DB30171E
:10184A000343DB0175DD2575DC2575D84453F8FEA5
:09185A0053F7FEE4F56DD2E8221B
:101A3400E56D30E002FF22E4F56E756D03EF25E0FD
:071A4400F572D2DD7F0222E2
:1019CC00E56D30E002FF22E4F56E156F756D05EFE5
:0B19DC0025E04401F572D2DD7F0222FD
:061BA80020DBFDAF6D2201
:0D002600156FAF6E056E74772FF8E6FF22A0
:0C1B68007477256EF8EFF6056E156F22FD
:0E1B3200E4F5847585FFF592F5A475A5FF22F4
:071B9A00EE3395E0FDFC2293
:1018B000C212C214C211D2A2C2A0C2A1E4FDFF1280
:1018C0001956E4FD7F011219567F0812125D7F043C
:0318D00002125DA4
:10195600EF146011047016BD0104C2A78002D2A75D
:0E196600A2A7921322BD0103C2A622D2A6227E
:10125D00EF14B40800505C90127275F003A4C583AE
:10126D0025F0C5837302128A0212900212970212A0
:10127D00A30212A50212A30212AF0212B7D2127567
:10128D00190122C212A21392A722D214751A057D3A
:10129D00017F010219568005C211C28722C211D2E7
:1012AD008722D211D28775180122C2A47F0112168E
:0412BD00D7D2A422BE
:1015EF00301212D5190F30A707C2A775191E800523
:1015FF00D2A7751946E51AD39400400CD51A09C223
:10160F0014E4FD7F01121956301111D5180E3087D1
:0D161F0006C28775180522D28775181E2295
:10191600C374039FFE1392A0EEA2E192A1AF80CF03
:0F1926005480CFED547FCF4FCF8F80C2A2D2A27B
:01193500228F
:0617AA008B428A438944D2
:1017B000E4FCCFECCF7D201219160CBC04F4E4FC41
:1017C000AB42AA43A9448C82758300120722FD60B4
:0B17D0000ACFECCF1219160CBC04E588
:0117DB0022EB
:041182008F828E8347
:10118600121B9AE47B0F7A27F9F8C31208C05003A2
:1011960090270FAF82AE83121B9A7B197AFC79FFD8
:1011A60078FFD31208C0400390FC19E4F531741B94
:1011B6002531F8E4F60531E531B405F2AE83AF82A8
:1011C600121B9A7B007A00791B120D36E51E701AE7
:1011D600753103741A2531F8E6FF741B2531F8C6FC
:1011E600EFC6D531EE751B2080E27B007A00791BB5
:0311F6000217AA33
:1019740046554C4C0050524F47005A4C4F47004D6F
:0E1984004F44310076322E30005472696700F5
:101A4B00E6FE08E6FFE4FCFD78CA02090778CA1235
:071A5B0008FB78C202091428
:030013000218F5DB
:1018F500C0E0C0D075D010200E0CAF8DEFAD8BF5CC
:101905005EEDF55FD20E758D00758B00D0D0D0E001
:01191500329F
:0216D7008F4141
:1016D900E4F542F543C3E5439541E54294005023BF
:1016E900900000AF82AE83E4FCFD7B207A4EF9F8CE
:1016F900D31208C04003A380EA0543E54370D60529
:031709004280D249
:01170C0022BA
:0E1B40007BFF7A1979741217AA7F0A0216D752
:0F1B1500D20B301506121B40C20B22121667228C
:05000E00C20B02169F69
:101A620078CE12092000000000121A5878CA120912
:061A72002000000000222C
:10003600121B32121B7E1218B07F041216D720979D
:10004600127BFF7A1979791217AA7F011214E7D267
:10005600AF80FE20960912049A1211F912095F7AEE
:1000660019797E12048F7A19798312048F7BFF7AAD
:100076001979881217AA7F041216D7E4FF1214E71B
:1000860012049A7F011216D71211F9120019C21A18
:1000960012162C7F011216D7E4F560F56112001ACC
:1000A600A2969208A2979209E4F52478C61209202E
:1000B60000000000E4F52578CE120920FFFFD8F1F4
:1000C60078C212092000000000E4F55578CA12092A
:1000D6002000000000C20DC20BC20CE4F565F566F7
:1000E600F526F527F55EF55FC20EF562C20FF55CE3
:1000F600F55DF563F564F52078ABE624FE600B1438
:10010600600C2402700AD2018006D2068002D20058
:1001160078ACE624FE6007047006D2028002D2079D
:1001260078ADE624FE600B14600C2402700AD2033C
:100136008006D2048002D205300113C20178A5E6FA
:10014600FF7E007C007D641207838E5C8F5D301A13
:10015600FDC21A300C33A208309601B3400BA20937
:10016600309701B3400302023B30961230970FC21C
:100176000CE4F565F5667F0412125DE4F555A2966A
:100186009208A297920902023B209605209702D276
:1001960010309656309753301031C21078C212087C
:1001A600FBEC4D4E4F78CE700C120920000000007B
:1001B600121A5880101209200000000078C2120995
:1001C6002000000000D209D2088024789CE6601F37
:1001D6000566E56670020565D394B8E565940B403F
:1001E6000ED20C7F0512125D8005E4F565F566A258
:1001F60008309601B3501FA2969208309618201028
:1002060015C201E5556007E4F5557F06800575556D
:10021600017F0712125DA209309701B35017A2970A
:10022600920930971020100DB20B300B05121B15DA
:10023600800312000E1204A7E55D455C6014E55DBF
:10024600155D7002155CE55D455C7006200B0312BA
:100256001B15E56445636011E5641564700215635A
:10026600E5644563700312000E200E03020317C2F5
:10027600AFC20ED2AFE4855F30855E2FF52EF52D29
:10028600AF30AE2FAD2EAC2D7B107A27F9F81207C2
:10029600958F308E2F8D2E8C2DE4FB7A90F9F812E7
:1002A600152B8F308E2F8D2E8C2D78A3E66009C3EB
:1002B60074B89FFF740B9EFEE56214601624FE6000
:1002C6002024037049C3EF94B0EE9404500E756277
:1002D600018009D3EF9414EE9405403575620380CE
:1002E60030C3EF94B0EE94045027756201300006D7
:1002F600200B03121B15300305C203121A62300BC2
:1003060002D20F7BFF7A19798D1217AA8003E4F5C2
:10031600620525E525C394055003020489E4F52505
:10032600FB7A0079281218638E298F2AE528640241
:10033600600302048978C6120907E8C0E0E9C0E054
:10034600EAC0E0EBC0E0789BE6FDAF2AAE291214C6
:1003560011D0E0FBD0E0FAD0E0F9D0E0F8EB2FFFC7
:10036600EA3EFEE93DFDE83CFC78C6120914052488
:10037600E524C39405500302048978C61208FBE4F9
:100386007B05FAF9F812152B78C612091478C612ED
:1003960008FB78C2120907C3EF9BFFEE9AFEED99A0
:1003A600FDEC98FC78C612091478CE1208FB78C6C4
:1003B600120907D31208C0400A78C61208FB78CE85
:1003C600120914E555600A78D0E6FE08E68E2BF58C
:1003D6002C78C8E6FE08E68E29F52AE5556006AFB4
:1003E6002CAE2B8004AF2AAE29121182300B4E059B
:1003F60027E52770020526C3789A96E526189640C3
:100406003CE4F526F5277F0312125D300D0DE52934
:10041600FF120016AF2AE52A12001620151A78A434
:10042600E6600C300F097F007E8212110AC20FAF00
:100436002AAE2912110A8005121B40C20B78C61279
:1004460008FB78CA12091478C612092000000000B9
:10045600E4F524300405C204121A6230061178A7A6
:10046600121A4BD31208C04006200B03121B15307C
:10047600071178A9121A4BC31208C05006300B0395
:0904860012000E1215EF020154E0
:10048F007BFF1217AA7F041216D722D2AF1219E7D9
:08049F00C2177F7012183A2207
:1018D300444C0021536967005A4C4F47004D4F4415
:1018E3003100322E30004D617920313920323030D1
:0218F3003400BF
:1013C000AF39AE38AD37AC36EC4D4E4F22EF24FF7F
:1013D000F539EE34FFF538ED34FFF537EC34FFF531
:1013E0003622E475392075384EF537F53622E47526
:1013F0003901F538F537F53622FDFCAB39AA38A9A5
:1014000037A836C30208D675330075340075359792
:0114100022B9
:1004A700121B4EEF70030206D27F0412125DE4F5B1
:1004B70055C20CF565F5661219AFEF12093906C674
:1004C7002406CF2A06245204ED61055B6305AE6559
:1004D70005F96C05FF7205FC73062874069B760602
:1004E7009378000006D27BFF7A1879D31217AA12E5
:1004F70013E2121B4EEF700A1213C060051213CDE0
:1005070080F01213C070030206D21219AF8F321295
:1005170014A2E4F5391213F2E47F06FE1213F95020
:100527000A121A8D8F321206D380ED121A8D8F326E
:10053700E53264806016E53264816010120016129D
:100547001A8D8F321200167531018003E4F531E5FB
:100557003170D8221214071213EEF5321213C0604D
:10056700241213E2121B4EEF700A1213C060051219
:1005770013CD80F01213C060031206EC0532E5328A
:10058700C3941840D71213C0601A7897B6AB070800
:10059700B6CD030206CC7BFF7A1879D61217AA7F4D
:1005A7000A0216D7020690E4FFFE121A01E4F53993
:1005B7001213F2E4FF7E081213F95033121A8D8FCB
:1005C70031E539540FFFE4FEFDFCFBFAF9F8C312DD
:1005D70008D6700F121B91AE38AF39121B047F205B
:1005E700120016AF31121A1B7F201206D380C402E5
:1005F70006C3B20D220212C1121407E4F532AB335F
:100607000535E535AA347002053414F9120709FFD8
:100617001200160532E532C3941840E22243A208BD
:10062700227533007534007535751213EEF53212E5
:1006370013C060241213E2121B4EEF700A1213C08C
:1006470060051213CD80F01213C060031206EC058B
:1006570032E532C3940240D71213C0602CAE75AF97
:1006670076EE3395E0FDFC78CA120907C3EF9BF5D8
:100677003DEE9AF53CED99F53BEC98F53AAF3D78B0
:10068700A1E53CF608EFF6803C02170D7F04121235
:100697005D0213187A1879DB1207007A1879E012CD
:1006A70007007F761200167BFF7A1879E5121AF198
:1006B700121B917BFF7A1879E9121AF1021B91E458
:0B06C70078A1F608F602180D12145D71
:1006D20022120016E5392401F539E43538F538E4FB
:1006E2003537F537E43536F536221219AFAB33AA72
:1006F20034A935853282758300EF120761227BFFB0
:07070200121AF1121B9122F3
:0A1B7E00E4F5955396BF53A27F22B1
:10162C005389F0438901538FFE758C70E4F58A530E
:10163C00B8FD53B7FDD2A9D28C53890F438990536F
:10164C008FEFF58DF58B4391105392EF53B8F75301
:0B165C00B7F7D2ABD28ED28AD2AA22FE
:03000B00021B884D
:091B8800D21A758C70758A0032C6
:03001B00021BA124
:071BA100758D00758B003209
:101AB5000D0A003031323334353637383941424337
:041AC500444546004E
:101AC900AF54AB48AA49A94A055422AF47AE46AD1F
:041AD90045AC4422B2
:1014E7005387BF75985053877FE4F5BABF0105430B
:1014F700A240800353A2BFE4F5BD75BE30F5BF75AA
:10150700BD035391FE4392014391025392FDC21BC7
:1015170053B8EF53B7EF43B81078C0F618F678C151
:04152700F6D2AC222A
:030023000217764B
:10177600C0E0C0D075D01030981E78C0E6C3940F74
:10178600501418E60624AFF8A69978C00618E6C3E2
:10179600941040027600C298309904C299C21BD0B8
:0417A600D0D0E0328D
:08000300201BFDD21B8F992286
:1019360078C0E6D39400401508E60624AFF8E6FF23
:0F19460078C01608E6C394104005E4F6227F002F
:01195500226F
:03001600020003E2
:1019AF007F207E4E78C0E67010D3EF9400EE940047
:0C19BF004007EF1F70EE1E80EB1219367F
:0119CB0022F9
:101AF100120709FF600C120016740129F9E43AFA81
:031B010080EE2251
:0E1B4E0078C0E6D3940040037F01227F00227E
:101A1B00CEEFCEEE54F0C4540F901AB893FF1200D1
:091A2B0016EE540F93FF020016A1
:101B0400CDEFCDCCEECCEEFF121A1BCFEDCF021AE7
:011B14001BB5
:091B91007BFF7A1A79B5021AF102
:0E0D36008F478E468D458C448B488A49894AEA
:100D4400E4F554EC4D4E4F7017E94A4B70057F3073
:100D5400020016121AC98F827583007430020E596C
:100D6400121AD6EC33502AE54A4549454870077FA4
:100D74002D120016800D121AC98F82758300742DEE
:100D8400120761121AD41208B28F478E468D458C11
:100D940044755301754E00754DCA754C9A754B3B9D
:100DA400E4FFFEFDFCAB4EAA4DA94CA84BD31208A0
:100DB400D65003020E44121AD4A84B1208208F52A4
:100DC4008E518D508C4FEC4D4E4F7004E553702373
:100DD400E5522430FFE54A4549454870051200169E
:100DE400800EAE54121ACB8E82758300EF12076107
:100DF400E4F553AF4EAE4DAD4CAC4BAB52AA51A93A
:100E040050A84F120795C8ECC8C9EDC9CAEECAC3A9
:100E1400E5479FF547E5469AF546E54599F545E5E5
:100E24004498F544AF4EAE4DAD4CAC4BE47B0AFA5E
:100E3400F9F81208208F4E8E4D8D4C8C4B020DA468
:100E4400E549454A45486010AB48AA49A94A855432
:080E540082758300E4120761BE
:010E5C002273
:100B8A000134C35001DBBF68028BBB800344B798B2
:100B9A000407B3B004D5AFC805A9ABE00689A7F826
:100BAA000775A410086DA02809719C400A819858FD
:100BBA000B9F94700CCA90880DE98CF90E048CA0D6
:100BCA000EA88AAC0F4D88B80FF786C410A184D03E
:100BDA00115182DC120580E812BB7EF413747D0089
:100BEA0014307B0C14F2791815B8772416807530F6
:100BFA00174B733C1819714818ED6F5419C46D607E
:100C0A001AA16B6C1B7E69781C6167841D4A65900A
:100C1A001E37639C1F2561A8201A5FB421125DC08C
:100C2A00220D5BCC230E59D8241557E4251F55F005
:100C3A00262F53FC27425208285B501429764E204F
:100C4A002A9B4C2C2BC04A382CEE48442E1E465068
:100C5A002F55445C308F426831D1407433173E803F
:100C6A0034633C8C35B13A98370938A4386636B0C3
:100C7A0039C734BC3B2D32C83C9D30D43E0F2EE0E0
:100C8A003F882CEC41062AF8428D29044418271083
:100C9A0045AB251C4741232848E121344A861F4099
:100CAA004C311D4C4DE21B584F9C1964515D177015
:100CBA005323157C54EF138856C4119458A20FA0DD
:100CCA005A830DAC5C6D0BB85E6009C4605807D0DE
:100CDA00625A05DC646203E8667301F4688A0000FC
:100CEA006AA1FE0C6CB8FC186ECFFA2470E6F830D4
:100CFA0000000000000000000000000000000000EA
:100D0A0000000000000000000000000000000000D9
:100D1A0000000000000000000000000000000000C9
:0C0D2A00000000000000000000000000BD
:1015B00075F004E538A4248AF582E5F0340BF58350
:1015C000E49322FE740193FF75F004E538A422F53C
:1015D00083C37401939FFFE4939EFEE4228F398EB0
:0F15E000388D378C36228F358E348D338C3222F6
:101ADD00C3EF9DEE9C400AD3EF9BEE9A50037F011E
:041AED00227F002232
:040E5D008E368F3707
:100E6100E4F5381215B0FC740193FD1215C8248EF7
:100E7100F582E5F0340BF583E493FA740193FBAF4B
:100E810037AE36121ADDEF7003020F4D1215B01294
:100E910015C3248EF582E5F0340B1215CF8F3C8EED
:100EA1003BF53AF5391215C82490F582E5F0340B7B
:100EB100F583E4931215C3248CF582E5F0340B120B
:100EC10015CF8F408E3FF53EF53DAD3EAC3D12084E
:100ED100B28F408E3F8D3E8C3DAE36AF37E4FCFD88
:100EE100EEC0E0EFC0E01215B0FE740193FBCAEE54
:100EF100CAD0E0FFD0E0FEC3EF9BFFEE9AFEED9477
:100F010000FDEC9400FCAB40AA3FA93EA83D1207AE
:100F110095AB3CAA3BA93AA83912152BC8ECC8C914
:100F2100EDC9CAEECACBEFCB1215C8248CF582E508
:100F3100F0340BF583E493FE740193FFE4FCFDEBC5
:100F41002FFFEA3EFEED39FDEC38FC220538E5388D
:0D0F5100C3946A5003020E64E4FFFEFDFC31
:010F5E002270
:01001A0022C3
:10136E001215DDAB39AA38A937A836E8C0E0789F48
:10137E00E6FE08E6FFE4FCFDD0E0F8120795121534
:10138E00DD780E1208E71215DD78A1E6FE08E6FFFD
:10139E00EE3395E0FDFCE5392FF539E5383EF538AD
:1013AE00E5373DF537E5363CF536AF39AE38AD3776
:0213BE00FC220F
:021411008D311B
:10141300120E5D1215E612136E1215E6E531146015
:101423001C14702DE47FE87E03FDFCAB35AA34A9C0
:1014330033A832120795E47BE87A0B800CAF35AE04
:1014430034AD33AC32E47B03FAF9F812152B1215E1
:09145300E6AF35AE34AD33AC3226
:01145C00226D
:10070900BB010689828A83E0225002E722BBFE02EE
:09071900E32289828A83E4932221
:10072200BB010CE58229F582E5833AF583E022508C
:1007320006E92582F8E622BBFE06E92582F8E222D6
:0D074200E58229F582E5833AF583E49322F0
:10074F00BB010689828A83F0225002F722BBFE0189
:02075F00F32283
:10076100F8BB010DE58229F582E5833AF583E8F0CE
:10077100225006E92582C8F622BBFE05E92582C87A
:02078100F22262
:10078300EF8DF0A4A8F0CF8CF0A428CE8DF0A42E8A
:02079300FE2244
:10079500E88FF0A4CC8BF0A42CFCE98EF0A42CFC03
:1007A5008AF0EDA42CFCEA8EF0A4CDA8F08BF0A481
:1007B5002DCC3825F0FDE98FF0A42CCD35F0FCEBE0
:1007C5008EF0A4FEA9F0EB8FF0A4CFC5F02ECD39A5
:0F07D500FEE43CFCEAA42DCE35F0FDE43CFC2212
:1007E40075F008758200EF2FFFEE33FECD33CDCCCC
:1007F40033CCC58233C5829BED9AEC99E58298404F
:100804000CF582EE9BFEED9AFDEC99FC0FD5F0D62B
:10081400E4CEFBE4CDFAE4CCF9A88222B800C1B955
:100824000059BA002DEC8BF084CFCECDFCE5F0CB93
:10083400F97818EF2FFFEE33FEED33FDEC33FCEBCC
:1008440033FB10D703994004EB99FB0FD8E5E4F987
:10085400FA227818EF2FFFEE33FEED33FDEC33FC74
:10086400C933C910D7059BE99A4007EC9BFCE99A68
:10087400F90FD8E0E4C9FAE4CCFB2275F010EF2FAD
:10088400FFEE33FEED33FDCC33CCC833C810D707AD
:100894009BEC9AE899400AED9BFDEC9AFCE899F8E8
:0E08A4000FD5F0DAE4CDFBE4CCFAE4C8F9227B
:10152B00C2D5E830E70FB2D5E4C39BFBE49AFAE4EB
:10153B0099F9E498F8EC30E717B2D5121561120857
:10154B0020E4C39BFBE49AFAE499F9E498F880034E
:10155B0012082030D50DE4C39FFFE49EFEE49DFDF1
:04156B00E49CFC22DE
:0E08B200C3E49FFFE49EFEE49DFDE49CFC2257
:1008C000EB9FF5F0EA9E42F0E99D42F0EC6480C8AF
:0608D00064809845F0224F
:1008D600EB9FF5F0EA9E42F0E99D42F0E89C45F078
:0108E60022EF
:1008E700E86010ECA2E713FCED13FDEE13FEEF1327
:0408F700FFD8F02214
:0C08FB00E6FC08E6FD08E6FE08E6FF2229
:0D090700E6FB08E6F908E6FA08E6CBF82260
:0C091400ECF608EDF608EEF608EFF6220F
:10092000D083D082E493F608740193F6087402939E
:09093000F608740393F6740473D5
:10093900D083D082F8E4937012740193700DA3A34D
:1009490093F8740193F5828883E473740293686061
:06095900EFA3A3A380DF61
:00000001FF
